:08373F0033302E312020200060
:06346B00C110C10FC10EEB
:10216900E4FFFE7D807C3F121048020B2A90031386
:102179001210C190000912100C900005121054029F
:10218900089312103C120BD5123737E4FF12373778
:10219900121A1BD2FA22854A4B85494A854849AF0A
:1021A9005712363B8F482290031A121048E4FFFE5B
:1021B9007D807C3F02088F7FCD7ECC7DCC7C3D121B
:1021C9001048020893120893797F7843E4FBFA02D6
:1021D9000A8DE4FFFEFD7C409003161210480209A7
:1021E9008485454685444585434485574322900265
:1021F900F91210E1900005120D65FF900006120D0D
:1022090065FD900004020D65783FE4FBFAF90209C7
:1022190084121084E4FFFE227B017A0279E690029F
:10222900F91210E1900003120D65FF900202E06FB0
:1022390022E543540FC454F0FFF0E54354F0C4546D
:102249000F4F22FFEC3EA3F0A3EFF09003BEE0FE98
:10225900A3E07802229003130210C19003E1E0FC8D
:10226900A3E0FD22C286D286E50825E02278411244
:102279000A8D783FE4FBFAF9020893FEE433A3F0F0
:10228900A3CEF09003D9E0C313FEA3E02290022D60
:1022990002103C90031E12108490031A02103CFF96
:1022A900E433FEF0A3EFF0D394FFEE940022121072
:1022B90084AF03AC07E4020BA1A804A905AA06ABE5
:1022C90007221210C190000502100CE548540FC4F2
:1022D90054F0FFF0E548223E9003E5F0A3EFF090BB
:1022E90003E522E0FEA3E0FFEE4F24FF92872212CE
:1022F900291C90027E1210C1E94A22E4FBFA798076
:10230900783F020B2AAD07AC06ED4C229002480239
:10231900103C12103C9003030210849002640210D6
:102329003C7FCD7ECC7DCC227BCD7ACC783D02081A
:012339009310
:031A0F00C295225B
:031A1500D2952245
:0D36AE00A295E43370047F0180027F0022AA
:102A59009003E1EEF0A3EFF0D3943FEE648094800D
:102A6900501C122264EC120B9C7B8B7AEC798178D6
:102A7900C21209847B007A40799C784580661222CB
:102A890064D39480EC648094805019EC120B9C7B85
:102A99005F7A98793778C11209847B647A2F79CA69
:102AA90078448040122264D394C0EC6480948050AE
:102AB90019EC120B9C7B787AB4790178C0120984DD
:102AC9007BD77AB279CF7843801A122264EC120B41
:102AD9009C7B887A4679B778BE1209847B5C7A8FA9
:082AE90079C078421208932223
:1034E40075A4CD75F22FE4F5F3F5A5F5A675F407EB
:0A34F40075D4C075E10675E24422AC
:1036280075BC4475E88075BA1F75D108E4F5BB43CD
:03363800E608227F
:0A37100075A14075F809E4F5A22246
:10366E0075DA2175DB2175DC2175DD2143E610222B
:09372E00E4F5B1F5A975B283229E
:102AF1007592107593EC75910443E680900244122F
:102B0100109000000000900248121090437F0000D6
:102B110090024C121090437F0000900254121090CA
:102B2100412000009002581210904396000090023C
:102B31005C1210903F800000900260121090000023
:102B41000000900264121090437F0000900268120E
:102B51001090437F000090027012109041200000FD
:102B6100900274E4F0A37464F0A31210903F80000B
:0C2B71000090027A1210903F80000022B9
:0B36FA0075CA8F75CBFFD2CAD2AD227B
:10361200758850758922758E0C758AAE758CAE755B
:063622008BC7758DC72265
:1032D400E4F5D975FF8075EF02121A15900240F0DB
:1032E400A3F0A3F0A304F090023F7480F012372EF1
:1032F4001234E412362812371012366E1236FA12CD
:053304002AF10236125F
:10311500FEE4339003E3F0A3CEF09003E3E0C313A2
:0D312500FEA3E09003E313FFEEF0A3EFF034
:103132007E0090023DE0FCA3E0FD120DC67C007D06
:10314200FF120E2D7C007DFF120DC6E024FFFD90C4
:09315200023DE034FFFC120DD82F
:01315B002251
:10363B00EF131313541FFEEF5407C43354E04EFF24
:01364B00225C
:10340500EF4E700C1221EAAF431231328F35800E28
:10341500EF64014E700812219F1231328F3612323D
:023425009D22E6
:1031A10012230E70191221EA9003D812223AF02547
:1031B100431222849003D912312B8F358022ED6482
:1031C100014C701C12219F9003D81222D412224567
:1031D100F0254812228413FF9003D912312D8F3626
:0331E10012329D0A
:0131E40022C8
:1033910012230E700E1221EAE54325441231158FD6
:1033A100358012ED64014C700C12219FE5482549CE
:0833B1001231158F3612329D16
:0133B90022F1
:0426CC00AB07AA06A8
:1026D000EB4A705C1221EA9003BB12223AFFF0E54C
:1026E000431313543FFEA3F0E5435403C433335460
:1026F000C04EF9F0E54325E025E0FEA3F0E54354A4
:10270000C0FDC4131354034EF0E5432FFFE433FE22
:10271000E97C002FFFEC3EFEE02F12224CCEC313CB
:10272000CE13D8F9FF9003BE12312D8F35022796B4
:10273000EB64014A706012219F9003BB1222D412F5
:102740002245FFF0E5481313543FFEA3F0E548543B
:1027500003C4333354C04EFEF0E54825E025E0FDC8
:10276000A3F0E54854C0C4131354034DFDF0EFFB30
:10277000E5482BFBE433FAEE7E002BFFEE3AFE7CBD
:1027800000EF2D12224CCEC313CE13D8F9FF9003C5
:09279000BE12312D8F3612329D6C
:01279900221D
:102DE90012230E70311221EAE5432544FFE433FE34
:102DF9007A00EF2545FFEA3EFEEF2546FFEA12225B
:102E0900E0122257CEC313CE13D8F9FF9003E5126F
:102E1900312D8F358035ED64014C702F12219FE5DE
:102E2900482549FFE433FE7C00EF254AFFEC3EFECE
:102E3900EF254BFFEC1222E0122257CEC313CE131B
:0E2E4900D8F9FF9003E512312D8F3612329D1D
:012E57002258
:1030C4009002391210904000000090023DE4F0A3F9
:1030D4007402F07BFF7A34790590027E1210E1E4E9
:1030E400F508F543F544F545F546F547F548F54942
:1030F400F54AF54BF54CF537F538753901F53A7560
:103104003B01753C01753D02F53E753F0275400279
:013114002298
:10291C00E4900242F0A3F090023FE0FFC3947C509D
:10292C0008900242E4F0A304F0E4900240F0A3F01B
:10293C00EFD394834008900240E4F0A304F090029B
:10294C00421222ECC286D2869002401222EC122253
:10295C006D2437F8E6FFB40204D2878002C287C226
:10296C0086D286EFB40104D2878002C28712226D10
:10297C002437F8E67004D2878002C28712226D24B5
:10298C0038F8E6FFB40204D2878002C287C286D22E
:10299C0086EFB40104D2878002C28712226D2438DC
:0F29AC00F8E67004D2878002C287C286D28622E4
:101194001232D490020230B0057432F080037433FA
:1011A400F0900202E0FF1236C843F6011230C41276
:1011B40035661234AAE5B05404F52530B10343254D
:1011C4000112368E757400757532C20DD2AF1229B4
:1011D4001CD212301010900202E0FF7BFF7A3779A4
:1011E4003F12306CC210300F0A900202E0FF123539
:1011F40099C20FE528700302128B14605B24FD6012
:10120400030212851235CB0508E508C39405400393
:10121400E4F508E50814600F1460141460191460F0
:101224001E2404702280207BFF7A3179A1801E7BEA
:10123400FF7A33799180167BFF7A2679CC800E7BF6
:10124400FF7A2D79E980067BFF7A34790590027E56
:101254001210E112291C8029300E1AA20DB3920D2E
:10126400300D0AC219121A0F1235CB8014121A1536
:1012740012368E800C1236AEEF6006123763121AE5
:101284001512291CE4F52820110302146CC21190D4
:10129400022512103C90022912108490022112108F
:1012A4003C90022512108490021D12103C900221E1
:1012B40012108490021912103C90021D12221A7D01
:1012C4007F7C439002141221E4120BD512363B1298
:1012D40022BC1221D1900219121084900210121013
:1012E4003C90021412108490020C12103C900210D4
:1012F40012108490020812103C90020C1210849078
:10130400020412103C900208121084AC57E4120B31
:10131400A11221D1900204121084AC5EE4120BA13C
:10132400C004C005C006C007AC0EE4120BA1D00374
:10133400D002D001D0001221CE90022D1210849040
:10134400022D122169600C400A90022D1210903F68
:10135400800000AC5DE4120BA1C004C005C006C04F
:1013640007AC0DE4120BA1D003D002D001D00012BF
:1013740021CE900231121084900231122169600C46
:10138400400A9002311210903F800000AC5BE412DE
:101394000BA1C004C005C006C007AC0CE4120BA12D
:1013A400D003D002D001D0001221CE900235121009
:1013B4008490023FE55FF0E4FFFE7D807C3F900275
:1013C40035122170600C400A9002351210903F8053
:1013D4000000AC5CE4120BA1C004C005C006C00749
:1013E400AC0BE4120BA1D003D002D001D000120840
:1013F400937BBC7A7479397841120A8D7840122231
:101404007D90023912221A7DC07C4190023912214A
:1014140070600C400A90023912109041C000009094
:10142400023912103C120BD590023DEEF0A3EFF0FE
:10143400E57545746008E5751575700215747D13BE
:10144400E4FF121A307D147F01121A307D0D7F02E1
:10145400121A307D0C7F03121A307D0E7F04121A8B
:10146400307D0F7F05121A307B017A0279E612343F
:1014740027EF70030211D59002E8E01210EA14EF8E
:101484000415000514B91414A11614AE1714BE1AC9
:1014940014D81B14E31D14E91E0000151AD20DD232
:1014A4000E121A0F1235CB02151A121A15C20D128A
:1014B400368E02151AD20E02151A7B017A0279E6CB
:1014C4009002F61210E1120D4CFE900202E0FF6E43
:1014D40070448005900202E0FF1235E402151A12EE
:1014E400375602151A12375D02151A122221702678
:1014F400300D1B1221F7FB122D788012122221705D
:1015040015300D0A1221F7FB122B7D1215C2900221
:1015140002E0FF1235B2200D0302146C9002E8E0E1
:1015240014601A24FA602214604D24066003021425
:101534006C121595900381F012376380341215955F
:10154400900381F01215C280281215AB12220BFDF4
:10155400900005120D65FBC0039002FC1210C190AF
:101564000006120D65900329F0D003122C86121583
:10157400CC12371A02146C1215AB12220BFD900018
:1015840005120D65FB12279A1215CC12371A021494
:011594006CEA
:1015950012365D7B017A0279E69002F61210E1902F
:1015A5000003120D652212365D7B017A0279E69001
:1015B50002FC1210E1900003120D65FF221234AAFD
:1015C50012369E12291C221234AA12369E12291C8A
:0115D50022F3
:102E5800E5B05404F52430B103432401E524652585
:102E6800600CE5246525F526752703852425E527C7
:102E780060291527E5277023E52630E011E5242091
:102E8800E00C9002827401F0A37490F0D214E5264D
:102E980030E208E52420E20375280430142090026B
:102EA8008274FFF5F0120E6330B105752801C21463
:0F2EB800900282E07002A3E07004C214D21022D4
:031A12000237692F
:05376900C2CFD2FF32C7
:061A1B00E5A120E7FB221B
:08373700E5A120E7FB8FA322AE
:031A2D000215D6C9
:1015D600C0E0C0F0C083C082C0D075D000C000C0DB
:0D15E60001C002C003C004C005C006C0075C
:1015F30053917FE50925599003C01222A840099011
:1016030003C0E4F0A374FFF01223159002441221E7
:101613007090025C50091210903F80000080071206
:101623001090BF800000900244121048C000C00117
:10163300C002C0039003C0E0FEA3E0FF122A597961
:10164300A078401221D5C004C005C006C00790028F
:101653005C12103C9002541221E4D003D002D0015A
:10166300D000120A8DD003D002D001D0001208930B
:1016730090024412221AFDFC90025C122170601049
:10168300400E9002441221C0900248122170401B68
:10169300E4FFFEFDFC90025C122170503D90024875
:1016A3001221C0900244122170502FAF57EFC31381
:1016B300FBEF30E004EB4480FB12231590024C1245
:1016C30022B79002481210849002441210489002EC
:1016D300481218A990025412108490024412231B3A
:1016E30012231590030712108490024C12103C121F
:1016F300286690025012221A7D7F7C43900250127A
:101703002170600C400A900250121090437F000039
:10171300E4FFFEFDFC900250122170500A9002502B
:1017230012109000000000C2FA7F30123737900287
:101733005012218BE50A255A9003C21222A84009B0
:101743009003C2E4F0A374FFF0122324900260120A
:10175300217090027650091210903F80000080079C
:10176300121090BF800000900260121048C000C0A9
:1017730001C002C0039003C2E0FEA3E0FF122A5996
:10178300E4FBFA79A07840120A8DC004C005C006B4
:10179300C00790027612103C9002701221E4D0032D
:1017A300D002D001D000120A8DD003D002D001D0D4
:1017B3000012089390026012221AFDFC9002761226
:1017C30021706015401312232A7C3D900260122180
:1017D300C89002641221704020E4FFFEFDFC9002D9
:1017E30076122170504212232A7C3D90026412210A
:1017F300C8900260122170502FAF57EF25E0FBEF26
:1018030030E704EB4401FB1223249002681222B751
:1018130090026412108490026012104890026412C5
:1018230018A990027012108490026012231B1223D5
:101833002490030712108490026812103C12286649
:1018430090026C12221A7D7F7C4390026C122170ED
:10185300600C400A90026C121090437F0000E4FF7A
:10186300FEFDFC90026C122170500A90026C121063
:101873009000000000C2FA7F3112373790026C12D9
:0B188300218B122E5875E89075BB01F8
:10188E00D007D006D005D004D003D002D001D000AE
:10189E00D0D0D082D083D0F0D0E03212103C1208DB
:0E18AE008F1236D5E4FBFAF97841120A8D222A
:031A21000219D7D0
:1019D700C0E0C0D075D000C000C007C2EDE5BB6055
:1019E70019AFBB74522FF8A6BE75E890E5BBB414C7
:1019F7000575BB00800905BB800585BE67D211D080
:081A070007D000D0D0D0E0327E
:10329D00C2FA7F32123737AF35122191C2FA7F331E
:1032AD00123737AF36122191C2FA7F341237379069
:1032BD000203E0FF122191C2FA7F351237379002D7
:0732CD0018E0FF122191221D
:10367E001222F8600A89828A83E4FFFE1211142254
:10364C001222F8600B89828A837F017E001211148A
:01365C00224B
:061D08009003131210E12C
:101D0E007F9A7E997D997C3E90022D122170503CD7
:101D1E00E4FBFA79807840122296120A8D794C12E1
:101D2E00233112225E900001121054120B2A9003DE
:101D3E00136010400E1222CBE4FBFA798012227649
:101D4E00021E6B122179122211021E6B1222967B39
:101D5E009A7A997999783E120B2A600250547F9A9A
:101D6E007E997D197C3F90022D12217050441222D3
:101D7E005E90000112100CC004C005C006C0071210
:101D8E00232A7CBD90022D1221C81222C2D007D068
:101D9E0006D005D004120B2A900313500C1222CB3E
:101DAE00E4FBFAF912227680061221791222110230
:101DBE001E6B1222967B9A7A997919783F120B2A0A
:101DCE00600250317433FFFEFD7C3F90022D1221D4
:101DDE0070502212217612225E90000D1221851271
:101DEE00225E900011122185E4FBFA7980783E1272
:101DFE000984021E6B1222967433FBFAF9783F1295
:101E0E000B2A600250287FCD7ECC7D4C7C3F900209
:101E1E002D122170501812217612225E90000D1292
:101E2E00218574AAFBFAF9783E120984802F1222BA
:101E3E00967BCD7ACC794C783F120B2A60025017E4
:101E4E007466FFFEFD7C3F90022D12217050081229
:101E5E002176122211800612225E1222CE90031AD1
:101E6E001210847FCD7ECC7D4C7C3F9002351221AA
:101E7E00E479CC12233190031612221AFD7C3F9086
:101E8E00031612217050331221DB90031A1221E433
:101E9E0012229C90031E1221C8122304506F12218D
:101EAE00DBC004C005C006C0071221B0D003D002AB
:101EBE00D001D000120A8D021F0F9003161221B30B
:101ECE0078401222131222C21222A2120A8D12225C
:101EDE009C90031E1221C812230450319003161237
:101EEE0021B3E4FBFAF97840120984C004C005C09E
:101EFE0006C0071221B0D003D002D001D0001209C3
:101F0E00841222C21221B690031E12108490023146
:101F1E001221B31221E1C004C005C006C007900310
:101F2E001E12103C9002311221E4D003D002D001D7
:101F3E00D00012089390032212221A7D7F7C4390C8
:101F4E0003221221E4120BD512225EEF120D921211
:021F5E00329DB2
:011F6000225E
:031A240002300885
:10300800C0E0C0F0C083C082C0D075D000C000C08E
:1030180001C002C003C004C005C006C00730D805FF
:10302800C2D812367E30D905C2D912364C30DA0BE6
:10303800C2DA7B017A027903121D0830DB0BC2DB8E
:103048007B017A027918121D08D007D006D005D066
:1030580004D003D002D001D000D0D0D082D083D009
:04306800F0D0E03292
:10348B00E475F001120E7985F082F5832275B7A5EC
:0F349B0075B7F18F828E8322EEF0A3EFF0A3229C
:1034FE00A2AFE433FCC2AF758F01123498EDF0E445
:09350E00F58FAF04EF24FF92AF2A
:013517002291
:10358000A2AFE433FDC2AF758F03123498E4F0F5B7
:083590008FAF05EF24FF92AF9D
:013598002210
:1031E5009003C41234A3ECF0A3EDF0EB4A603190E8
:1031F50003C4E0FEA3E0FFA3E0FCA3E0F5828C831B
:10320500E0FD1234FEEB1B70011A9003C6E475F065
:1032150001120E639003C4E475F001120E6380CBB6
:013225002286
:08374700E4900000F0A3F02261
:1033BA00900000E0FEA3E0FF123580900000E0FEDE
:1033CA00A3E0FF7C007D027B007A021231E5E490E3
:0633DA000000F0A3F02248
:0A2D0100A9059003AFEEF0A3EFF078
:102D0B00EE54FEFE900000E0FCA3E0FD7002EE6CC2
:102D1B006042ED4C60031233BA9003AFE0FEEE5409
:102D2B00FEFE7F00900000F0A3EFF09003B1123491
:102D3B00A37400F0A37402F07E029003B112348BE3
:102D4B00E493FD9003B312348BEDF0EF1F70011E73
:102D5B00EF4E70E69003AFE0FCA3E0FDEC5401FCFA
:0C2D6B0074022DF58274003CF583E9F041
:012D77002239
:1032650090039A1234A31210E190039F74FFF5F0B6
:10327500120E7945F0602090039AE475F001120E64
:1032850079AFF0FE90039CE475F0011210CA120D9F
:083295004CFD122D0180D22234
:10347100420287000042028C000042028E0000C11D
:0534810016C117C11582
:10315C0090028EE475F001020E63D3900288E09029
:10316C0002879400E06480948022E0FEA3E0249027
:10317C00F58274022290028EF0A3F02274FFF5F017
:10318C00020E63E0F5C2C2C5C2C49002D322FCE5B4
:05319C00F064404C222C
:10336700C217C216E4900287F0A3F090028CF0A374
:10337700F0900290F012318190028AF0A37440F02D
:0A338700E4900289F09002D0F022D9
:0D36BB0075C19043E6019002857401F02274
:10365D0043C140E5C120E5FB123367E4900285F0DC
:01366D00223A
:0A371A0053C1BF9002857401F02234
:0D36C800AE071236BB900286EEF0023367AB
:1033E000E49003E7F0A3F0301702FF222016FDD28D
:1033F000179002D1E4F0A37410F09002D4EFF0E43F
:04340000A3F07F01B5
:0134040022A5
:10333B0030170A9002D1E07002A3E070037F0022E5
:10334B009002D11231889002D5E0FE04F074D62E93
:0C335B00F582E43402F583EFF07F0122DC
:0B370500301707C217D216123724221B
:0A372400E5C120E5FBC2C4D2C522B6
:102EC7009003A21210E1900285E07002FF229003A6
:102ED700A5E0FE6005D3941040037F00221233E083
:032EE700EF604950
:102EEA00E49003A7F09003A5E0FF9003A7E0FEC3D8
:102EFA009F501F9003A21210C18E82758300120D7B
:102F0A0065FF12333BEF7002FF229003A7E004F043
:102F1A0080D3E49002D0F01237059003A6E0700344
:092F2A002016FD9002D0E0FF2208
:032F33007FFF22FB
:0B29BB009003C81210E19003CBEDF078
:1029C60012316650037F002290028E1231763EF558
:1029D60083E0FF12315C12319A700312318190024A
:1029E6008A12315FE4FE9003CBE0FDEEC39D5035C5
:1029F600EEC39F503090028EE0FC1231783CF58396
:102A0600E0FD9003C81210C18E82758300ED120D91
:102A1600A412315C12319A700312318190028A122B
:102A2600315F0E80C1EEC39F501412315C12319A91
:102A3600700312318190028A12315F0E80E7900294
:102A4600871231889003CBE0FEEFC39E50028002CE
:022A5600AF06C9
:012A5800225B
:0C36E20012316640047F0180027F00224C
:031A180002233A6C
:10233A00C0E0C0F0C083C082C0D075D000C000C069
:03234A0006C007C3
:10234D00C21AE5C054FE1210EA241B08241B0A23EE
:10235D00E20C23E20E248E10248E1223E82223F3A6
:10236D002823F32A23E82C23E82E23D5C02395C256
:10237D002387E02387E200002499C2159002D4122E
:10238D00318F74FFF002249B9002D3E0FFB4FF0B5A
:10239D009002D512318FE4F002249B9002D5E0FE1D
:1023AD00EFC39E50179002D3E0FF04F074D62FF5C3
:1023BD0082E43402F583E0F5C202249BD2C490027C
:1023CD00D0E4F0C21602249B9002D074FDF0D2C569
:1023DD00C2C402249B9002D374FFF0D215C2C4C2B2
:1023ED00C1D2C502249BE5C26007900286E0B5C24A
:1023FD000E900284E4F0C2C5C2C4D2C102249BC2B5
:10240D00C4C2C1301503022493C2C502249BD390CC
:10241D00028BE090028A12316E405C12318890027C
:10242D0084E07006E5C2F0E004F0900284E0FFC3A2
:10243D0090028BE09F7480F890028AE0648098503F
:10244D0004C2C1804990028C1231763EF583E5C2FB
:10245D00F090028C12315FFEE5F064404E700690F4
:10246D00028CF0A3F0900284E014F07006900287C5
:10247D00123160D2C1801790028974FFF0C2C18001
:10248D000DC2C4301508C215D2C58002D21A301A39
:10249D001053C17F43C180C2C5C2C4C2C1C21AC2DA
:0324AD0016C2C094
:1024B000D007D006D000D0D0D082D083D0F0D0E0EA
:0124C00032E9
:051A2700E5C15420FFA1
:011A2C002297
:103518007B01E49003B9F0227422F0A3EFF0A32218
:0A3528007B01E49003B9F07D04225A
:0B3226009003B51210E19003B8EDF02A
:10323100E49003BAF09003B51210C19003B8E09086
:1032410003A5F09003B9E09003A6F0E4FF122EC7A6
:10325100EFB4FF0D9003BAE0FE04F0EEC394034017
:03326100D47E0018
:013264002247
:063427009003DB1210E12E
:10342D007E007F007D101211169003DB1210C17DFE
:0B343D00101229BBEF7002FF227F017C
:013448002261
:10306C009003481235207413F0120D4C90034BF062
:10307C00900001120D6590034CF0900002120D654A
:10308C0090034DF0900003120D6590034EF09000EC
:10309C0004120D6590034FF0900005120D6590031E
:1030AC0050F0900006120D65900351F07A037948A8
:0830BC001235187D0A023226CC
:103599009003CC1235207403F0A374FFF07A0379F9
:0935A900CC1235187D0402322613
:1035E4009003D0123520741CF0A374FFF07A037991
:0735F400D012352802322637
:1035B200E49003D4F0A3EFF0A3740AF0A3EFF07A3F
:0935C2000379D4123528023226E7
:1033090074FFF5F0020E63EFF0A3ECF0A3EDF0A368
:103319000210E1D2C1C2C4D2C5E4FF9003EAF0228F
:10332900E50F8510F0020E63E025E044A0F5C27FA9
:0233390003226D
:07374F0043C14053E6FE22D6
:0625D800900332123310E3
:1025DE0090033B7403F0A374E8F0E5C120E5FB1211
:1025EE00331C30C0FDE5C054FEFE244070030226AD
:1025FE007E24FE601A24E2600924FE600524E202B5
:10260E002686C2C5EF7077900332123331806FEF9A
:10261E00B4030A900333E0F5C27F058061EFB40581
:10262E000B900333A3E0F5C27F068052EF64067071
:10263E002D90033AE0900335700875F0011210CA20
:10264E0080031210C1120D4CF5C2900338123309DB
:10265E00900338E07002A3E070247F078020EFB46F
:10266E000706D2C47F0980169003EA7405F0800E27
:10267E009003EA7402F080069003EA7401F0EFB45E
:10268E000904C2C080329003EAE0FE6406600EEEDA
:10269E00B4021290033B12330945F06008D2C5E430
:1026AE009003EAF0FF9003EAE06008C2C5D2C4C20C
:0D26BE00C08005C2C00225F0E5C120E5FB8B
:0126CB0022EC
:0618BC00900352123310EC
:1018C20090035A7403F0A374E8F0E5C120E5FB121B
:1018D200331C30C0FDE5C054FEFE1210EA18F800B9
:1018E20019813819568A1989C0191FC218FBE018C4
:1018F200FBE2000018F8021991C2C5EF70099003CB
:1019020052123331021997EF640160030219979062
:101912000352E025E044A1F5C27F048078EFB403CE
:101922000A900353E0F5C27F05806AEFB4050B907D
:101932000353A3E0F5C27F06805BEFB40606D2C56F
:101942007F018051EFB404047F0280499003EA745E
:1019520005F08041900355E475F0011210CAE5C20A
:10196200120D92900358123309900358E07002A3AB
:10197200E070087F09C2C1D2C4801A7F028016902B
:1019820003EA7406F0800E9003EA7402F080069077
:1019920003EA7401F0EFB40904C2C080329003EA92
:1019A200E0FE6406600EEEB4021290035A1233098E
:1019B20045F06008D2C5E49003EAF0FF9003EAE044
:1019C2006008C2C5D2C4C2C08005C2C00218D4E534
:0419D200C120E5FB50
:0119D60022EE
:1024C100900366EFF09003691210E1900367ECF05E
:0324D100A3EDF088
:1024D400751100543FF512543F604BC3744095127C
:1024E400FFE49511FE90036CE0FCA3E0FDC39FECB8
:1024F4009E50068C0F8D1080048E0F8F101225AF06
:1025040060037F022290036712332990036EE07008
:102514000690036A123329C390036DE09510F0907E
:10252400036CE0950FF090036CE0F50FA3E0F51059
:10253400D3E5109400E50F9400406DE5109440E558
:102544000F9400500F1225AF60037F0222E4F50FB1
:10255400F51080DC900366E0FFA3E0FCA3E0FDA39C
:102564001210C1900338E4F0A37440F090036EE0BD
:1025740090033AF01225D89003EAE060037F022228
:1025840074C02510F51074FF350FF50F900367E440
:1025940075F040120E6390036EE0709490036A75B8
:0A25A400F040120E630225347F00A0
:1025AE0022900366E0FFA3E0FCA3E0FDA31210C19E
:1025BE00900338E50FF0A3E510F090036EE0900362
:0A25CE003AF01225D89003EAE0224B
:1035FB00900358E4F0A304F01218BC9003EAE060C7
:07360B00037F01227F002272
:103532009003E9EBF07B017A0379E990036CE4F004
:0A354200A304F0E4A3F01224C12258
:10344900C007900390E0FFA3E0900358CFF0A3EFEB
:10345900F0D0071218BC9003EAE060037F01227FD5
:0234690000223F
:10354C00C007900398E0FFA3E090036CCFF0A3EFCB
:0A355C00F0E4A3F0D0071224C1220E
:102FA200F9F8120EAA900344021084900340121002
:102FB20084E47FFF7EFFFDFC900340021048754FC2
:102FC200007550017551007552012290033DE024B5
:102FD20009F8E6FF2290033EE0FEA3E0FFD394004F
:102FE200EE648094802290034402103C90034002DD
:102FF200103C90033DE0FF2468F8E6223395E0FDA3
:06300200FC7810020FF93A
:10368E00D206D205D204D203D202D201122FC02208
:10369E00C206C205C204C203C202C201122FC02258
:071A300090033DEFF0AB0550
:101A3700C2AFC200122FF79003A8F0FD74532BF822
:101A4700E6F9C39DFCE4940090033EF0A3CCF0308C
:101A5700074A90033EE0FCA3E0FDC3EC648094805A
:101A6700502B746E2FF8E67002760390033DE0FF6B
:101A7700246EF816E6707B746E2FF8760174532B7C
:101A8700F8E6FE74682FF8A606D2008065D3ED94B9
:101A970004EC648094804051C2078040122FD740E5
:101AA7002E90033DE0246EF8E67002760390033D26
:101AB700E0FD246EF816E67039746E2DF876017421
:101AC700532BF8E6FC74682DF8A604D2008023C3D4
:101AD700EF94FCEE6480947F500FD20790033DE0B3
:101AE7002468F8A601D200800990033DE0246EF82F
:101AF700E4F6E57545746003021D05200003021D29
:101B07000590033DE0FD2409F8E6FE74A92DF58252
:101B1700E43403F583E0FDEDFFE4FCFD90034012A0
:101B27001084122FD75003021BC5EE122FFE122F5F
:101B3700A7122FE8C006C0079003A8E0FFC374FFF1
:101B47009FFFE49400AB07FAE4F9F8D007D0061238
:101B57000F35122FA7900344121048C000122FCD43
:101B6700C374FF9FFFE49400FEE4FCFDD000122F36
:101B7700A4122FCD9003A8E0D39F900344400A12EC
:101B8700103CE47B407A01800712103CE47BC0FAEA
:101B9700122FA2122FBAC000122FE87810120FE6E8
:101BA700D000120E8F122FADD3120FD55003021C87
:101BB7005F9003401210900000FFFF021C5F90032C
:101BC7003EE0FEA3E0FFC3E49FFFE49EFE122FFE6C
:101BD700122FA7122FE8C0079003A8E0FBE4FAF939
:101BE700F8D007120F35122FA7900344121048C0E0
:101BF70000122FCDE4FCFDFED000122FA4122FCD32
:101C07009003A8E0C39F900344500A12103CE47B62
:101C1700407A01800712103CE47BC0FA122FA2120F
:101C27002FEEC004C005C006C007122FE8781012B7
:101C37000FE6A804A905AA06AB07D007D006D0056A
:101C4700D004120E9C122FADD3120FD5400A900369
:101C57004012109000000000122FEE90033DE0FBB1
:101C670024A9F582E43403F583EFF0122FEE780808
:101C7700120FE690034012108474092BF8E6FFE474
:101C8700FCFDFE122FBAC3120FD56012122FEE9071
:101C9700033DE02409F8A6071235CB12291C3007AB
:101CA70024122FF4FE2404FDE433FC74092FF8E614
:101CB700FFD39DEC6480F874809840028015EFC3D1
:101CC7009E50388023122FF4FE74092FF8E6FFD3B5
:101CD7009E400CE4F54FF550F5517552018014EE16
:101CE70024FCFEEFC39E5013754F00755001E4F5B9
:101CF70051F552754D2E754EE08003122FC0D2AFAD
:011D070022B9
:04348600410382007C
:102C0300900374E075F007A42401F582E4343AAF2D
:102C13008222E475F001120E63900376E475F001ED
:102C2300020E63FE7B007A00790890039FE4F0A311
:102C33007407F022AFF0FEE0FCA3E0F5828C83E49E
:102C430093FD22900370F0A3EFF0E4900376F0A3DA
:102C5300F022EFF0A3EDF0A3EBF0A2AFE433A3F087
:102C6300C2AF2275F007A42401F9743A35F0FA7B58
:102C7300FF22E475F001020E79FDEDFFEEF0A3EF04
:032C8300F0E42258
:06375D00E4900382F0225B
:073756009003827401F022D0
:102F36009003DE7403F0E4A3F0FFA3F01237477E9C
:102F46003A7F007A0379DE122F941233BAE4F50839
:102F5600FF74092FF8E4F60FEFB406F5E49003DFEB
:102F6600F09003DFE0FFC3941E5012EF122C0712FD
:102F76002C261232659003DFE004F080E41233BAA7
:0E2F86007E3A7FD37A0379E0122F940233BA99
:0E2F94007B0190039FE4F0A304F0123265224B
:1035CB00201915300E0D300D0D900382E07007D2CF
:0935DB000F8003121A0FD219220D
:10356600903AD3E493F46009903A00E493640360DC
:0A35760003122F36E4900381F022C7
:1034AA00900381E0FFC3941E5013EF122C66780834
:0E34BA007C007D007E007F07120D26C21922C5
:1034C800900381E0C3941E50121237479003811273
:0C34D8002C06122C261232651233BA2288
:063763001234C8C2192255
:052C8600900327EDF0B2
:102C8B00900329E004F090032CEFF0A3EBF09003FA
:102C9B0027E0FF90032CE0FED39F5059EE122C0738
:102CAB0090032EF0A3EFF090032D122C069003301F
:102CBB00F0A3EFF0E490032AF0A3F0900330122C72
:102CCB007590032E122C37122D0190032E122C1FF0
:102CDB0090032A122C1FC390032BE0940790032A16
:102CEB00E0940040D61233BA90032CE004F0A3E03A
:052CFB0004F0022C9919
:012D000022B0
:05279A0090036FEDF05B
:10279F00900374EFF0A3EBF090036FE0FF900374DE
:1027AF00E0D39F4003022865A3122C06122C4690FB
:1027BF000376E0FEA3E0FFC39407EE9400501A9057
:1027CF000370122C3A74832FF582E43403F583EDF2
:1027DF00F0900370122C1580D6122C03900372F018
:1027EF00A3EFF0900375122C06122C469003701273
:1027FF002C75900372122C37122D01900372122C2C
:10280F0015C3900377E09407900376E0940040DCC3
:10281F00122C03900372122C49900376E0FCA3E074
:10282F00FDC39407EC9400501D900372122C75AFEA
:10283F00F0FE74832DF582E43403F583E0FD122D51
:10284F0001122C1C80D31233BA900374E004F0A34E
:06285F00E004F00227A7CF
:012865002250
:032B7D0090035C66
:102B8000122C5512374F90035DE0FE90035CE090ED
:102B90000364122C7C900360F090035EE0FF9003CE
:102BA00064E0FCA3E0FD7B017A037983900390123B
:102BB0002C30123449900364E475F007120E6390D0
:102BC0000360E0122C66A31210E1123747900361F4
:102BD0001210C1AE02AF017B017A037983122C2D52
:102BE0001232651233BA900360E004F0E0C3941E21
:102BF00040A7900202E0FF1236C890035FE024FF76
:022C000092AF91
:012C020022AF
:032D78009003784D
:102D7B00122C5512374F900379E0FE900378E090B8
:102D8B00037D122C7C90037CF090037CE0FFC394BA
:102D9B001E503AEF122C07FE90037FF0FAA3EFF0D0
:102DAB00FB90037AE0FF90037DE0FCA3E0FDA90319
:102DBB007BFF900398122C3012354C90037DE475F9
:102DCB00F007120E6390037CE004F080BC900202CB
:0D2DDB00E0FF1236C890037BE024FF92AFAA
:012DE80022C8
:101F61000000000000000000000000000000000070
:101F71000001000100010001000100010002000256
:101F81000002000200030003000300030004000438
:101F9100000500050005000600060007000700080F
:101FA100000800090009000A000A000B000B000CE0
:101FB100000D000D000E000F000F001000110011A8
:101FC1000012001300140014001500160017001869
:101FD1000019001A001A001B001C001D001E001F22
:101FE10000200021002200230024002500270028D2
:101FF1000029002A002B002C002D002F0030003179
:10200100003200340035003600380039003A003C17
:10201100003D003E004000410043004400460047AF
:102021000049004A004C004D004F0050005200543E
:10203100005500570058005A005C005E005F0061C7
:102041000063006500660068006A006C006E007045
:1020510000710073007500770079007B007D007FBF
:10206100007F00810083008500870089008B008D3F
:10207100008F009000920094009600980099009BB8
:10208100009D009F00A000A200A400A600A700A937
:1020910000AB00AC00AE00AF00B100B200B400B5BF
:1020A10000B700B800BA00BB00BD00BE00C000C14F
:1020B10000C300C400C500C700C800C900CA00CCE5
:1020C10000CD00CE00CF00D100D200D300D400D586
:1020D10000D700D800D900DA00DB00DC00DD00DE2B
:1020E10000DF00E000E100E200E300E400E500E6DB
:1020F10000E700E700E800E900EA00EB00EB00EC94
:1021010000ED00EE00EE00EF00F000F100F100F252
:1021110000F300F300F400F400F500F500F600F61A
:1021210000F700F700F800F800F900F900FA00FAEA
:1021310000FB00FB00FB00FC00FC00FC00FC00FDC0
:1021410000FD00FD00FD00FE00FE00FE00FE00FEA1
:1021510000FF00FF00FF00FF00FF00FF00FF00FF86
:0821610000FF00FF00FF00FF7A
:0C36EE0012103C02088F9002FF021048EE
:062866009002FF12108435
:10286C009003071210489002FF1236EE1236D5E490
:10287C00FBFA7980783F120B2A600840069003031C
:10288C0002103C1236F49003071236EE90030B1232
:10289C0010841236F49003031236EE90030B1210D0
:1028AC0048120A8D90030F121084E4FFFE7D7F7C8A
:1028BC004390030F121048120984120BD5C3EE6417
:1028CC008094805003E4FEFFD3EF94FFEE64809479
:1028DC008040047E007FFFEF25E0FFEE33FE746145
:1028EC002FF582741F3EF583E493FE740193FFFD74
:1028FC00AC06EC120B9CE4FBFA797F7843120A8D40
:0F290C0090030B1210481209841236F41208932C
:01291B002299
:03000000020800F3
:03000300021A03DB
:03000B00021A06D0
:03001300021A09C5
:03001B00021A0CBA
:03002300021A0FAF
:03002B00021A12A4
:03003300021A1599
:03003B00021A188E
:03004300021A1B83
:03004B00021A1E78
:03005300021A216D
:03005B00021A2462
:03006300021A2757
:03006B00021A2A4C
:03007300021A2D41
:0C080000787FE4F6D8FD7581750208478A
:10088C00020C41E86480F8E933E83360110460F04D
:10089C00ED33EC337009E8FCE9FDEAFEEBFF2204D2
:1008AC0060DED3EB9FEA9EE99DE8C2E78CF0C2F7CD
:1008BC0095F0400CE8CCF8E9CDF9EACEFAEBCFFB99
:1008CC00120C0C85D0F05804700320D5B3E80470DA
:1008DC00075002B2D5020C4B92D5EC0460F7E4CC75
:1008EC00C0E0C398F8603B94186008400DD0E0FB62
:1008FC00020C23E4FBFAC9FC8028E830E406E4C9C6
:10090C00FBE4CAFCE830E305E4C9CACBFCE85407B5
:10091C006010F8C3E913F9EA13FAEB13FBEC13FCC0
:10092C00D8F130F52FC3E49CFCEF9BFFEE9AFEED63
:10093C0099FDD0E0FBEF4E4D4C701222DB03020C04
:10094C0048EC2CFCEF33FFEE33FEED33FDED30E7DE
:10095C00EB020C23EF2BFFEE3AFEED39FDD0E0FB62
:10096C0050130BBB0003020C4BED13FDEE13FEEF0B
:08097C0013FFEC13FC020C2335
:10098400EC4D6011E8497017ED33EC3304600DE46D
:10099400FCFFFEFD22E933E8330470F8020C411237
:1009A4000C0C58046009E4CC248150062850090238
:1009B4000C4B284003020C48C0E0EB4A7044B98059
:1009C40006D0E0FB020C37EF4E701CBD8008EBFF35
:1009D400EAFEE9FD80EBE98DF0A4FEE5F0020A6D84
:1009E400E9CDF9EAFEEBFFEF89F0A4FCE5F0CE894E
:1009F400F0A42EFFE435F0CD89F0A42DFEE435F00B
:100A04008067EF4E7005BD80D780C3EF8BF0A4AC38
:100A1400F0EE8BF0A42CFCE435F0F8EF8AF0A42C73
:100A2400E5F038FCE433CB8DF0A42CFCE5F03BF886
:100A3400EE8AF0A42CFCE5F038F8E433CF89F0A476
:100A44002CFCE5F038CF3400CE89F0A42FFFE5F07C
:100A54003EFEE433C98DF0A42EFEE5F039CD8AF0D4
:100A6400A42FFFE5F03EFEE43DFD33D0E0FB50074C
:100A74000BBB000F020C4BEC2CFCEF33FFEE33FEF0
:060A8400ED33FD020C231E
:100A8A00020C4BEC5D046005E859047003020C414A
:100A9A00120C0C580460F6EC4860F2EC7004FDFE8F
:100AAA00FF22C860DB2481C85009C398600250063F
:100ABA00020C489850CAF582E9294B4A7005AB8264
:100ACA00020C3775F0007C1A7880C3EF9BEE9AED22
:100ADA0099400DC3EF9BFFEE9AFEED99FDE842F0B7
:100AEA00DC23ACF0D0E0FFD0E0FED0E0FDAB82200A
:100AFA00E7101BEB60BAEC2CFCEF33FFEE33FEED94
:100B0A0033FD020C23E803F830E705C0F075F00066
:100B1A00EF2FFFEE33FEED33FD40B830E7C280AA77
:100B2A0074F8CC6480CCC86480C8F582046043C37E
:100B3A00EB9FF5F0EA9E42F0E99D42F0E89C45F011
:100B4A0060305018E5825FFFE582F42B5582FB5036
:100B5A00210ABA001D09B90019088016E5825BFB53
:100B6A00E582F42F5582FF50090EBE00050DBD0027
:100B7A00010CC3EB9FF5F0EA9E42F0E99D42F0E8D2
:0D0B8A009C45F06007CC4820E701B3EC2249
:100B970075F020800E75F010800575F0087D007ED9
:100BA700007F003392D530D503120FC7EC334010C6
:100BB700EF33FFEE33FEED33FDEC33FCD5F0ED22E2
:0E0BC700E5F0247EA2D513CC92E7CDCEFF221E
:100BD500EDD2E7CD33EC3392D524814006E4FFFE18
:100BE500FDFC22FCE4CFCECDCC24E0501174FF8077
:100BF500EDC3CC13CCCD13CDCE13CECF13CF047014
:070C0500F030D5DE020FC73D
:0D36D500ED33EC3360065004EC6480FC2201
:100C0C00E9D2E7C933E833F892D5EDD2E7CD33EC2E
:070C1C0033FC5002B2D522A7
:100C2300EC30E7100FBF000C0EBE00080DBD000432
:100C33000BEB6014A2D5EB13FCED92E7FD2274FFDE
:100C4300FCFDFEFF22E480F8A2D574FF13FC7D8037
:030C5300E480EF4B
:10080C00021194E493A3F8E493A34003F68001F25D
:10081C0008DFF48029E493A3F85407240CC8C333ED
:10082C00C4540F4420C8834004F456800146F6DFBC
:10083C00E4800B010204081020408090346BE47EAD
:10084C00019360BCA3FF543F30E509541FFEE493B1
:10085C00A360010ECF54C025E060A840B8E493A378
:10086C00FAE493A3F8E493A3C8C582C8CAC583CAA3
:10087C00F0A3C8C582C8CAC583CADFE9DEE780BE5B
:01348A000041
:100C5600E709F608DFFA8046E709F208DFFA803E80
:100C660088828C83E709F0A3DFFA8032E309F6086D
:100C7600DFFA8078E309F208DFFA807088828C83D5
:100C8600E309F0A3DFFA806489828A83E0A3F60889
:100C9600DFFA805889828A83E0A3F208DFFA804C63
:100CA60080D280FA80C680D4806980F2803380103A
:100CB60080A680EA809A80A880DA80E280CA8033A3
:100CC60089828A83ECFAE493A3C8C582C8CCC5831B
:100CD600CCF0A3C8C582C8CCC583CCDFE9DEE780EB
:100CE6000D89828A83E493A3F608DFF9ECFAA9F06A
:100CF600EDFB2289828A83ECFAE0A3C8C582C8CCC0
:100D0600C583CCF0A3C8C582C8CCC583CCDFEADED8
:100D1600E880DB89828A83E493A3F208DFF980CC3A
:100D260088F0EF60010E4E60C388F0ED2402B40433
:100D36000050B9F582EB2402B4040050AF232345DA
:060D46008223900CA6734D
:100D4C00BB010689828A83E0225002E722BBFE02A5
:090D5C00E32289828A83E49322D8
:100D6500BB010CE58229F582E5833AF583E0225043
:100D750006E92582F8E622BBFE06E92582F8E2228D
:0D0D8500E58229F582E5833AF583E49322A7
:100D9200BB010689828A83F0225002F722BBFE0140
:020DA200F3223A
:100DA400F8BB010DE58229F582E5833AF583E8F085
:100DB400225006E92582C8F622BBFE05E92582C831
:020DC400F22219
:100DC600EF8DF0A4A8F0CF8CF0A428CE8DF0A42E41
:020DD600FE22FB
:100DD800BC000BBE0029EF8DF084FFADF022E4CCFF
:100DE800F875F008EF2FFFEE33FEEC33FCEE9DECC8
:100DF800984005FCEE9DFE0FD5F0E9E4CEFD22ED0E
:100E0800F8F5F0EE8420D21CFEADF075F008EF2F57
:100E1800FFED33FD4007985006D5F0F222C398FD48
:050E28000FD5F0EA22E5
:100E2D00C2D5EC30E709B2D5E4C39DFDE49CFCEEE0
:100E3D0030E715B2D5E4C39FFFE49EFE120DD8C373
:100E4D00E49DFDE49CFC8003120DD830D507C3E46E
:060E5D009FFFE49EFE224F
:100E6300C5F0F8A3E028F0C5F0F8E582158270021A
:060E73001583E038F022B7
:100E7900A3F8E0C5F025F0F0E5821582700215832C
:060E8900E0C838F0E82289
:0D0E8F00EF2BFFEE3AFEED39FDEC38FC22B2
:0E0E9C00C3EF9BFFEE9AFEED99FDEC98FC2251
:100EAA00E88FF0A4CC8BF0A42CFCE98EF0A42CFCE7
:100EBA008AF0EDA42CFCEA8EF0A4CDA8F08BF0A465
:100ECA002DCC3825F0FDE98FF0A42CCD35F0FCEBC4
:100EDA008EF0A4FEA9F0EB8FF0A4CFC5F02ECD3989
:0F0EEA00FEE43CFCEAA42DCE35F0FDE43CFC22F6
:100EF90075F008758200EF2FFFEE33FECD33CDCCB0
:100F090033CCC58233C5829BED9AEC99E582984032
:100F19000CF582EE9BFEED9AFDEC99FC0FD5F0D60F
:100F2900E4CEFBE4CDFAE4CCF9A88222B800C1B939
:100F39000059BA002DEC8BF084CFCECDFCE5F0CB77
:100F4900F97818EF2FFFEE33FEED33FDEC33FCEBB0
:100F590033FB10D703994004EB99FB0FD8E5E4F96B
:100F6900FA227818EF2FFFEE33FEED33FDEC33FC58
:100F7900C933C910D7059BE99A4007EC9BFCE99A4C
:100F8900F90FD8E0E4C9FAE4CCFB2275F010EF2F91
:100F9900FFEE33FEED33FDCC33CCC833C810D70791
:100FA9009BEC9AE899400AED9BFDEC9AFCE899F8CC
:0E0FB9000FD5F0DAE4CDFBE4CCFAE4C8F9225F
:0E0FC700C3E49FFFE49EFEE49DFDE49CFC223B
:100FD500EB9FF5F0EA9E42F0E99D42F0E89C45F072
:010FE50022E9
:100FE600E8600FECC313FCED13FDEE13FEEF13FFE9
:030FF600D8F1220D
:100FF900E8600FEFC333FFEE33FEED33FDEC33FC56
:03100900D8F122F9
:10100C00BB010DE58229F582E5833AF58302103C9C
:10101C005007E92582F8021142BBFE07E92582F848
:10102C0002114EE58229F582E5833AF58302115AC5
:0C103C00E0FCA3E0FDA3E0FEA3E0FF2227
:0C104800E0F8A3E0F9A3E0FAA3E0FB222B
:10105400BB010DE58229F582E5833AF58302104848
:101064005007E92582F802116ABBFE07E92582F8D8
:10107400021177E58229F582E5833AF5830211842A
:0C108400ECF0A3EDF0A3EEF0A3EFF022DF
:10109000A8828583F0D083D0821210A71210A712E5
:1010A00010A71210A7E473E493A3C583C5F0C5830A
:1010B000C8C582C8F0A3C583C5F0C583C8C582C8AA
:0110C000220D
:0910C100E0FBA3E0FAA3E0F92230
:1010CA00F8E0FBA3A3E0F925F0F0E58215827002AF
:0710DA001583E0FA38F02253
:0910E100EBF0A3EAF0A3E9F02210
:1010EA00D083D082F8E4937012740193700DA3A395
:1010FA0093F8740193F5828883E4737402936860A9
:06110A00EFA3A3A380DFA8
:061110008A838982E4736A
:10111600EF4E6012EF60010EEDBB010B89828A83F0
:10112600F0A3DFFCDEFA2289F05007F709DFFCA9FD
:0C113600F022BBFEFCF309DFFCA9F02254
:0C114200E6FC08E6FD08E6FE08E6FF22D9
:0C114E00E2FC08E2FD08E2FE08E2FF22DD
:10115A00E493FC740193FD740293FE740393FF22DB
:0D116A00E6FB08E6F908E6FA08E6CBF822F5
:0D117700E2FB08E2F908E2FA08E2CBF822F8
:10118400E493F8740193F9740293FA740393FB22C1
:00000001FF
